:100000000C9461030C94A5030C94A5030C94A50314
:100010000C94A5030C94A5030C94A5030C94A503C0
:100020000C94A5030C94A5030C94590E0C942B0F5F
:100030000C94A5030C94A5030C94A5030C94A503A0
:100040000C94A5030C94E5220C94A5030C94A50331
:100050000C94A5030C94781C0C94A5030C94A50394
:100060000C94A5030C94A5030C94A5030C94A50370
:100070000C94A5030C94A5030C94A5030C94A50360
:100080000C94A5030C94A5030C94A5030C94A50350
:100090000C94A5030C94A5030C94A5030C94A50340
:1000A0000C94A5030C94A5030C94A5030A060F0653
:1000B000140619061E06230628062D063206980F7A
:1000C000BA0FA810BA0FA810FF0F2210A8107710AF
:1000D0008A105913591388138813BE13DE130F1592
:1000E0000F15E9130F159914991400150F150F1515
:1000F0000915A614A614A614A614A614A614A614CC
:10010000A614A614A614A614A614A614A614A6141F
:10011000A614B814C514CC14D314DD14012E022E69
:10012000012C022C0001E10135023502E10001350C
:1001300002350001E1012E022E012C022C02E10009
:1001400001E6012E022E02E6012C022C0001E10143
:1001500030023002E1012C022C0001E10164026452
:1001600002E100016402640001E60130023002E6AF
:10017000012C022C000000002200C001C002C003BC
:10018000C004C005C006C007C008C02E002D02373D
:10019000021E02045200002514140004001D00F485
:1001A00000387426141A0015001B00F5003771245E
:1001B000140900160006002B00C1002714130017B5
:1001C00000190036782D0031020A000700050000F2
:1001D00000230201541F020000360200003500C552
:1001E000003200000027020000490021140D000B1E
:1001F000000E000000240225020F00110010005024
:10020000004C002602180008004F0029002C00C3F3
:10021000001C000C005100C7002800C4002F001271
:1002200000520020022A001F14340033003802025A
:10023000520000241601000100010001000000012D
:1002400000010001000100010001000100010001A6
:1002500000010001003778251601000100010001AE
:1002600000010026160100010001003671010001A5
:100270000001000100010000000100010001000078
:1002800000010000002414010064000000010000CF
:100290000001002102010001000100000001000135
:1002A0000001000100010001000100010001000146
:1002B00000010001000100C8000100010001002E42
:1002C000140100C90001000100010001000100311A
:1002D00000010001000100035200000100010001C3
:1002E00000010001000000010001002000010001E8
:1002F000000100010001001F0001000100010001D8
:100300000001001E0001000100010001002202277F
:1003100000210001000100010001000100010000B6
:1003200000010001000100000001000000010001C7
:1003300000010000000100000001000100010001B7
:10034000004A00000001000100C200220026004A0D
:100350000001000100C60023004D00010001000162
:1003600000010024004E00010001000100010025F1
:10037000004B00010001000100010001000100012B
:100380000000000100010001000100010000000167
:100390000001002000010001000100010001001F18
:1003A00000010001000100010001001E0001000128
:1003B00000010001002202270021000100010001CC
:1003C0000001000100010000000100010001000027
:1003D0000001000000010001000100000001000018
:1003E0000001000100010001004A000000010001BD
:1003F00000C200220026004A0001000100CA0023BA
:10040000004D00010001000100010024004E000128
:100410000001000100010025004B00010001000166
:1004200000010001000100010000002200010001A4
:1004300000010001000000010001003C000100017A
:10044000000100010001003B00010001000100016A
:100450000001003A0001000100010001000100015B
:10046000003D000100010001000100010001000049
:100470000001000100010000000100000001000176
:100480000001000000010000000100010001000166
:1004900000301400000100010001003E0042000194
:1004A000000100010001003F0043000100010001C4
:1004B0000001004000440001000100010001004172
:1004C00000450001000100010001000100010001E0
:1004D00000000016034500720067006F0044006FC3
:1004E000007800200045005A000000160345007205
:1004F0000067006F0044006F007800200045005A3C
:100500000000000403090409026D00040100A0FAC0
:100510000904000001030101000921110100012269
:100520003F000705810308000A09040100010301D7
:100530000200092111010001224D00070582030874
:10054000000A090402000103000000092111010052
:10055000012236000705830308000A09040300018D
:100560000300000009211101000122390007058460
:10057000031000011201100100000008EDFE071336
:1005800001000102000105010906A101050719E0AA
:1005900029E7150025019508750181020508190153
:1005A00029059505750191029501750391010507CE
:1005B0001900297715002501957875018102C0057C
:1005C000010980A101850216010026B7001A010069
:1005D0002AB700751095018100C0050C0901A10121
:1005E0008503160100269C021A01002A9C02751040
:1005F00095018100C005010902A1010901A10005C1
:100600000919012905150025019505750181029536
:1006100001750381010501093009311581257F9597
:10062000027508810609381581257F9501750881B5
:1006300006050C0A38021581257F9501750881068B
:10064000C0C005010906A101050719E029E7150049
:10065000250195087501810295017508810105083C
:1006600019012905950575019102950175039101FF
:100670000507190029FF150025FF9506750881005B
:10068000C00000000000000000000000010204069D
:100690000A0F17202C3A4A5D71879DB3C7DAE9F536
:1006A000FCFFFCF5E9DAC7B39D87715D4A3A2C205F
:1006B000170F0A06040201000000000000000000FD
:1006C000000011241FBECFEFDAE0DEBFCDBF04B6BD
:1006D00003FE24C08091FB019091FC01A091FD01DB
:1006E000B091FE018730904BA740B04BB9F4109207
:1006F000FB011092FC011092FD011092FE0114BE4C
:1007000084B7877F84BF88E10FB6F8948093600038
:10071000109260000FBEE0E0FFE3099511E0A0E059
:10072000B1E0E8E5F9E402C005900D92A433B10709
:10073000D9F711E0A4E3B1E001C01D92AB3FB107CE
:10074000E1F70E949D0B0C94AA240C9400001092D7
:10075000B9008AE08093B800089594EA9093BC00B1
:100760009091BC0097FFFCCF9091B900987F983092
:1007700021F0903111F081E008958093BB0084E86E
:100780008093BC008091BC0087FFFCCF8091B900B2
:10079000887F883111F0803471F780E0089584E912
:1007A0008093BC008091BC0084FDFCCF08958093B1
:1007B000BB0084E88093BC008091BC0087FFFCCF25
:1007C0009091B900987F81E0983209F480E0089513
:1007D00084E88093BC008091BC0087FFFCCF8091AF
:1007E000BB00089580910101811115C080E40E9431
:1007F000AD038093010181110CC082E10E94D703F7
:1008000080930101811105C08FEF0E94D70380936F
:1008100001010E94CF0384B1807F84B985B1807FBC
:1008200085B98AB1837F8AB98BB1837F8BB93E98B2
:10083000469808950E94AF05809301010E94F2033B
:1008400080B38C7080BB81B3836F81BBA5E3B1E0C3
:10085000E3E4F1E08EE08E0F11921D928E13FCCF37
:100860000C949905BF92CF92DF92EF92FF920F9373
:100870001F93CF93DF9380910101882379F08091BA
:1008800034018F5F80933401811108C00E94AF054D
:1008900080930101811102C00E94410505E311E02E
:1008A000C0E0D0E0DD24D39482E0C82EEE24E394AF
:1008B000F12CC730D10500F580910101811164C090
:1008C00080E40E94AD0380930101811112C082E196
:1008D0000E94D7038093010181110BC0C7010C2E28
:1008E00001C0880F0A94EAF780950E94D70380938D
:1008F00001010E94CF0348C0CA30A1F028F4C830DB
:1009000059F0C93061F005C0CC3089F070F0CD30BD
:1009100089F0209A289810C0219A29980DC0229A0F
:100920002A980AC0239A2B9807C0529A01C0539A5A
:100930005B9802C03E9A469890EA9A95F1F79FB16B
:10094000799902C082E001C080E091709D25982BCA
:100950007C9902C084E001C080E0892B7D9902C0AF
:1009600038E001C030E0832B7E9902C020E101C055
:1009700020E0822B9FB19095991F9927991F9295FE
:10098000990F907E892B0FC080910101811149C080
:1009900080E40E94AD0380930101882379F1B12C9A
:1009A0000E94CF038B2DF8019081981719F0808356
:1009B000C09200010E94F20321960F5F1F4FCE30BC
:1009C000D10509F076CF80910001882361F1815033
:1009D00080930001882339F08FE99FE00197F1F7B8
:1009E00000C0000020C0A3E4B1E0E5E3F1E0CF01E6
:1009F000825F91919D938E13FCCF15C083E10E947D
:100A0000D703809301018111CACF81E40E94AD0315
:100A1000809301018111C3CF0E94E803B82EB094E6
:100A2000BFCF80E0C0CF0E943F0581E0DF91CF9132
:100A30001F910F91FF90EF90DF90CF90BF9008959E
:100A4000E82FF0E0ED5BFE4F8081089508950F934D
:100A50001F93CF93DF93C3E4D1E010E00C2F025F2C
:100A6000899190E00E94EE1B180F0C13F9CF812F93
:100A7000DF91CF911F910F910895089508950C94DF
:100A80003E0556985E9825982D9826982E9827987A
:100A90002F988FEF90E09093890080938800909337
:100AA0008B0080938A0090938D0080938C00259A10
:100AB0002D9A2FEF80E792E0215080409040E1F79F
:100AC00000C00000269A2E9A2FEF80E792E0215076
:100AD00080409040E1F700C00000279A2F9A2FEF46
:100AE00080E792E0215080409040E1F700C0000094
:100AF00025982D982FEF80E792E02150804090407C
:100B0000E1F700C0000026982E982FEF80E792E0D2
:100B1000215080409040E1F700C0000027982F98B6
:100B200056985E9825982D9826982E9827982F9855
:100B3000089589EA8093800089E080938100249859
:100B40002C983F988AB18F748AB96E98479A8BB166
:100B5000806B8BB9769A0E9441050C943D0580E22A
:100B6000809301018091510181110EC00E94A70361
:100B700081E0809351012FEF83ED90E3215080407D
:100B80009040E1F700C0000080E40E94AD03809334
:100B9000010181112EC00E94D703809301018111B0
:100BA00028C00E94D70380930101811122C08FE3E6
:100BB0000E94D7038093010181111BC00E94CF03C3
:100BC00080E40E94AD0380930101811112C08CE08A
:100BD0000E94D7038093010181110BC00E94D703AB
:100BE00080930101811105C08FE30E94D703809398
:100BF00001010E94CF03809101010895FC018281CF
:100C0000462F50E04930510590F5FA01EA5AFF4F5E
:100C10000C945A24882359F188E691E0089588239A
:100C200031F183E691E00895882309F18AE591E0A6
:100C300008958823E1F08DE491E008958823B9F0C8
:100C400080E491E00895882391F083E391E0089592
:100C5000882369F08EE291E00895882341F085E2CF
:100C600091E00895882319F08CE191E0089580E0E7
:100C700090E0089581E0089581E008950C943C0689
:100C800008950F931F93CF93DF938C01FC01C081D4
:100C9000D181CE010E94731ABE010E94EA06EC01C6
:100CA000B8010E943E06882309F48DC0F8018281B4
:100CB000882309F44AC080915D0181111FC0C431AD
:100CC000F0E5DF0709F051C00E94400681E0809303
:100CD0005D010E94421C90935C0180935B01109225
:100CE0005401109256011092550110925801109221
:100CF000570110925A011092590165C080915B0111
:100D000090915C010E944E1C883C910570F480918A
:100D10005401E82FF0E0EE0FFF1FEB5AFE4FD18396
:100D2000C0838F5F809354014EC0C43880E5D807DC
:100D300021F0C538D04501F13AC0F80182818823FD
:100D400041F01092520182E01EC0C438E0E5DE0797
:100D500059F580915201811106C086E20E94FD1171
:100D600086E20E94C51282E01CC0C438F0E5DF07AD
:100D700041F3C538D045D9F4F8018281882331F098
:100D80001092530180E20E9414131DC08091530100
:100D9000811106C087E20E94FD1187E20E94C51200
:100DA00080E20E941B130FC0C538D04529F381E0B3
:100DB0008093520180935301C801DF91CF911F911D
:100DC0000F910C943A0680E0DF91CF911F910F9123
:100DD0000895089596E0799FF001112494E5899F84
:100DE000E00DF11D1124E60FF11DEE0FFF1FE55779
:100DF000FE4F859194910895880F991FFC01EB5047
:100E0000F040859194910895880F991FFC01EB584B
:100E1000FE4F8591949108950F931F93CF93DF9385
:100E2000EC01811520E3920750F5C11580E2D80747
:100E300008F0C3C0CB3BD10590F4C83AD10508F007
:100E40006AC0C53AD10508F05BC0C430D10508F0CE
:100E5000D0C1219709F0CAC101E010E00AC2CF3F1A
:100E6000D10511F008F0C5C1C03FD10508F0A2C0FE
:100E7000CE01805E9109089708F4BBC1B7C1C130AB
:100E800090E5D90709F4A2C020F5C0318FE4D80756
:100E900070F4C11590E4D90708F094C0C11521E39E
:100EA000D20708F0A3C1DD278E01106CE2C1C11585
:100EB000D04509F09BC10E947A158FEF94E32CE096
:100EC000815090402040E1F700C000000E949D1C2E
:100ED000D0C1C11597E5D90758F4C03121E5D20733
:100EE00008F01CC1C43180E5D80708F475C07EC184
:100EF000CE0190578115904108F078C1DF7073C121
:100F0000C53AD10509F477C1C63AD10509F076C1D1
:100F100002E810E4AEC1C83AD10509F472C1C93A79
:100F2000D10509F471C1CA3AD10509F470C1CB3AAF
:100F3000D10509F46FC1CC3AD10509F46EC1CD3A9F
:100F4000D10509F46DC1C03BD10509F46CC1CE3A9D
:100F5000D10509F46BC1CF3AD10509F46AC1C13B8F
:100F6000D10509F469C1C23BD10509F468C1C33B8D
:100F7000D10509F467C1C43BD10509F466C1C53B7D
:100F8000D10509F465C1C63BD10509F464C1C73B6D
:100F9000D10509F463C1C83BD10509F462C1C93B5D
:100FA000D10509F461C1CA3BD10509F460C100E073
:100FB00014E45FC18E0110655CC1CE019F700E9478
:100FC000040758C1DF708E01106A53C18091DA01A5
:100FD00081608093DA014DC10E94421E811102C0DE
:100FE0000E94281E0E945F1E90E09093FB01809358
:100FF000FA01C23080E5D80721F48091FA018160BE
:1010000086C0C43090E5D90721F48091FA0182604E
:101010007EC0C63020E5D20721F48091FA018460B9
:1010200076C0C83080E5D80719F48091FA0127C04E
:10103000CA3090E5D90721F48091FA01806167C038
:10104000CC3020E5D20721F48091FA0180625FC0A4
:10105000CE3080E5D80721F48091FA01806457C032
:10106000C03190E5D90721F48091FA0180684FC022
:10107000C23120E5D20729F48091FA0184608860AA
:1010800046C0C33080E5D80721F48091FA018E7FF5
:101090003EC0C53090E5D90721F48091FA018D7FDB
:1010A00036C0C73020E5D20721F48091FA018B7F4A
:1010B0002EC0C93080E5D80719F48091FA0126C006
:1010C000CB3090E5D90721F48091FA018F7E1FC0C3
:1010D000CD3020E5D20721F48091FA018F7D17C031
:1010E000CF3080E5D80721F48091FA018F7B0FC0C3
:1010F000C13190E5D90721F48091FA018F7707C0BB
:10110000C331D04531F48091FA018B7F877F809382
:10111000FA018091FA010E94631EABC08D2F9927BE
:101120008F70992781309105D9F49E012370332760
:1011300002C0880F991F2A95E2F79C688E0144E04F
:10114000000F111F4A95E1F700271370802B912B98
:1011500053E0CC0FDD1F5A95E1F7C076DD272FC095
:101160008230910531F4DC2FCC278E01016F106A9B
:1011700080C08330910569F4CE018370992701E026
:1011800010E002C0000F111F8A95E2F7C8019C68A9
:101190000FC084309105B9F4CE018370992701E026
:1011A00010E002C0000F111F8A95E2F7C8019A688B
:1011B00023E0CC0FDD1F2A95E1F7C07ED7708C01AC
:1011C0000C2B1D2B56C08530910531F4DC2FCC271C
:1011D0008E01046F106A4DC0069709F04AC0CF71A6
:1011E000DD27DC2FCC278E01106243C000E010E029
:1011F00040C08E013EC001E810E43BC003E810E4AB
:1012000038C002EE14E435C009EE14E432C00AEE30
:1012100014E42FC005EB14E42CC006EB14E429C041
:1012200007EB14E426C00CEC14E423C00DEC14E42A
:1012300020C003E815E41DC00AE815E41AC002E95D
:1012400015E417C004E915E414C001E216E411C066
:1012500003E216E40EC004E216E40BC005E216E455
:1012600008C006E216E405C007E216E402C00AE27E
:1012700016E4C801DF91CF911F910F91089596E078
:10128000799FF001112494E5899FE00DF11D11244F
:10129000E60FF11DEE0FFF1FE557FE4F859194916C
:1012A000803E9105E0F4803C910558F5813391052D
:1012B00009F46FC048F48932910509F463C08A3299
:1012C000910509F46DC072C089339105E9F0823847
:1012D0009105D1F08533910509F44DC067C0833E77
:1012E000910581F138F4803E9105B9F0823E910577
:1012F000D9F05CC0863E910561F1873E9105A1F170
:1013000055C00E94FC0608952091FA0120FD02C0FC
:1013100021FF4CC080EE90E049C08091FA0180FF2F
:10132000F9CF89E390E042C08091FA0182FF0EC0BC
:101330008091FA0184FF03C080E090E037C083EE23
:1013400090E034C08091FA0182FFF2CF82EE90E00B
:101350002DC08091FA0183FF0BC08091FA0184FDBA
:10136000EBCF87EE90E022C08091FA0183FFF5CFAA
:1013700086EE90E01BC08091FA0185FF07C089E2EC
:1013800090E014C08091FA0185FFF9CF85E390E0E9
:101390000DC08091FA0186FF07C08AE290E006C086
:1013A0008091FA0186FFF9CF81E390E00E940C075B
:1013B000089508950C94D90980916E010895CF93F2
:1013C000DF9300D01F92CDB7DEB79C018091F10171
:1013D000843019F593E099833B832A839093E90045
:1013E0008FEF9091E800815095FD06C095ED9A959C
:1013F000F1F700008111F5CF8091E80085FF0DC065
:1014000040E050E063E070E0CE0101960E94490C9C
:101410008091E8008E778093E8000F900F900F90F6
:10142000DF91CF910895CF93DF9300D01F92CDB776
:10143000DEB72091F101243021F522E029839B833E
:101440008A8383E08093E9008FEF9091E8008150D8
:1014500095FD06C095ED9A95F1F700008111F5CF45
:101460008091E80085FF0DC040E050E063E070E04F
:10147000CE0101960E94490C8091E8008E778093FE
:10148000E8000F900F900F90DF91CF910895209179
:10149000F1012430F1F422E02093E9002FEF3091A4
:1014A000E800215035FD06C035ED3A95F1F7000012
:1014B0002111F5CF2091E80025FF0BC040E050E05E
:1014C00065E070E00E94490C8091E8008E7780937F
:1014D000E8000895CF93DF93EC019091F1019430EF
:1014E00009F046C080910C018823D9F080910D014C
:1014F0008823B9F09093E9008FEF9091E800815034
:1015000095FD06C095E19A95F1F700008111F5CFA0
:101510008091E80085FF2CC040E050E060E170E081
:1015200017C081E08093E9008FEF9091E80081502F
:1015300095FD06C095ED9A95F1F700008111F5CF64
:101540008091E80085FF14C040E050E068E070E062
:10155000CE010E94490C8091E8008E778093E800CC
:1015600080E1FE01AEE5B1E001900D928A95E1F7D0
:10157000DF91CF9108958091F001811109C00E94FF
:10158000DE0D0E943B0E8091E20084608093E200B9
:1015900008951092F001089508950C94D2220E94AB
:1015A000331C0E94D8220E94E1100C94DA0942E018
:1015B00061EC81E00E94580D42E061EC82E00E9403
:1015C000580D42E061EC83E00E94580D42E161EC6D
:1015D00084E00C94580D8091F301833009F455C0D8
:1015E00030F4813071F0823009F48EC008958A3071
:1015F00009F47AC08B3009F460C0893009F09CC0CE
:1016000020C08091F201813A09F096C08091E800F3
:10161000877F8093E8008091F6019091F701892BF4
:1016200021F460E18EE591E003C060E080E090E0AD
:1016300070E00E94940C8091E8008B778093E80022
:1016400008958091F201813209F076C08091F6010F
:101650009091F701009719F0039709F06DC0809100
:10166000E800877F8093E8008091E80082FD05C054
:101670008091F1018111F8CF5FC08091F1008093DA
:101680006E018091E8008B7753C08091F201813A1E
:1016900009F052C08091F6019091F701892B09F071
:1016A0004BC08091E800877F8093E8008091E8003C
:1016B00080FFFCCF80910C0136C08091F201813215
:1016C000D9F58091F6019091F701892BA9F58091C8
:1016D000E800877F8093E8000E948D0D8091F401DF
:1016E00080930C010C947A158091F201813221F5DE
:1016F0008091E800877F8093E8000E948D0D8091A3
:10170000F50180936F0108958091F201813AA1F46F
:101710008091E800877F8093E8008091E80080FF57
:10172000FCCF80916F018093F1008091E8008E776B
:101730008093E8000C948D0D089584B7877F84BF53
:1017400088E10FB6F89480936000109260000FBE9D
:1017500090E080E80FB6F894809361009093610068
:101760000FBE0E9430110E94DE0D0E943B0E809140
:10177000E20084608093E20078940E94C1100E948D
:10178000321182E091E00E94DC100E94C022809120
:10179000F101853069F40E94FA1B8091EF018823E2
:1017A000B1F30E94251C882391F30E94330CEFCFE4
:1017B0000E943811ECCF292F332723303105C9F08F
:1017C00064F42130310581F02230310509F043C045
:1017D0008DE690E027E035E042C021323105F1F09E
:1017E0002232310541F137C082E190E024E735E053
:1017F00036C099278130910541F08230910541F042
:10180000892B49F5E3E0F5E005C0EBEEF4E002C01A
:10181000E3EDF4E0849190E09F0121C06430D8F4BE
:10182000E62FF0E0EE0FFF1FEE5DFE4F20813181CD
:1018300089E090E014C0643070F470E0FB01EE0FBA
:10184000FF1FE65EFE4F20813181FB01EA5EFE4F05
:10185000808190E004C080E090E020E030E0FA0178
:1018600031832083089580E189BD82E189BD09B477
:1018700000FEFDCF8091D8008F7D8093D8008091AD
:10188000E00082608093E0008091E00081FDFCCF69
:101890000895CF92DF92EF92FF920F931F93CF9311
:1018A000DF93EC018B016A010E94AC0D811133C002
:1018B000C114D10439F0F60180819181081B190B04
:1018C000C80FD91FE12CF12C0115110519F18091D8
:1018D000E80085FD16C08091E8008E778093E800CF
:1018E000C114D10449F0F60180819181E80EF91EFE
:1018F000F182E08285E00FC00E94AC0D882321F3C5
:101900000AC089918093F10001501109FFEFEF1A8D
:10191000FF0ADACF80E0DF91CF911F910F91FF9006
:10192000EF90DF90CF9008952091F8013091F90168
:101930002617370748F06115710539F42091E80042
:101940002E772093E80001C0B90140E061157105D0
:10195000A9F12091F101222309F443C0253009F4B3
:1019600042C02091E80023FD40C02091E80022FD04
:1019700032C02091E80020FFE9CF4091F300209190
:10198000F20030E0342BFC01CF016115710559F0F4
:101990002830310540F481918093F1006150710944
:1019A0002F5F3F4FF1CF41E02830310509F040E093
:1019B0002091E8002E772093E800C8CF4111C9CFCD
:1019C0000AC08091F101882361F0853061F0809137
:1019D000E80083FD0AC08091E80082FFF2CF80E03A
:1019E000089582E0089583E0089581E008952091AC
:1019F000F8013091F9012617370748F06115710594
:101A000039F42091E8002E772093E80001C0B90155
:101A1000FC0120E06115710591F18091F1018823AD
:101A200009F440C0853009F43FC08091E80083FD8F
:101A30003DC08091E80082FD2FC08091E80080FFCA
:101A4000E9CF2091F3008091F20090E0922B611594
:101A5000710559F08830910540F424912093F100EC
:101A60003196615071090196F2CF21E0089709F093
:101A700020E08091E8008E778093E800CBCF2111A1
:101A8000CCCF0AC08091F101882361F0853061F0EC
:101A90008091E80083FD0AC08091E80082FFF2CFC8
:101AA00080E0089582E0089583E0089581E008953C
:101AB000982F973058F59093E900981739F0709166
:101AC000EC002091ED005091F00003C0242F762F00
:101AD00050E021FF19C03091EB003E7F3093EB00C6
:101AE0003091ED003D7F3093ED003091EB0031609F
:101AF0003093EB007093EC002093ED005093F000D6
:101B00002091EE0027FF07C09F5FD3CF8F70809397
:101B1000E90081E0089580E008958091F20187FF57
:101B200011C08091E80082FD05C08091F101811112
:101B3000F8CF11C08091E8008B770BC08091F10144
:101B4000882349F08091E80080FFF8CF8091E80079
:101B50008E778093E80008952091E4003091E500AD
:101B600095E64091EC00842F817040FF22C0809167
:101B7000E80080FD1CC08091F101882391F0853040
:101B800091F08091EB0085FD10C04091E4005091F0
:101B9000E5004217530729F39A01915011F784E0A9
:101BA000089582E0089583E0089581E0089580E03B
:101BB00008954091E80042FFDECF08950E944C0E48
:101BC0000E94540EE0EEF0E0808181608083E8EDB9
:101BD000F0E080818F77808319BCA7EDB0E08C9115
:101BE0008E7F8C9380818F7E80831092F001089588
:101BF0000F931F93CF93DF930E944C0E0E94540EBD
:101C0000C8EDD0E088818F77888388818068888359
:101C100088818F7D888319BC1092F1011092ED01AB
:101C20001092EF011092EE0100EE10E0F8018081B9
:101C30008B7F808388818160888342E060E080E0E0
:101C40000E94580DE1EEF0E080818E7F8083E2EE0D
:101C5000F0E0808181608083808188608083F801EA
:101C600080818E7F8083888180618883DF91CF919E
:101C70001F910F910895E8EDF0E080818F7E8083C1
:101C8000E7EDF0E080818160808384E082BF81E0C5
:101C90008093F0010C94F80DE8EDF0E080818E7FE8
:101CA00080831092E20008951092DA001092E10011
:101CB00008951F920F920FB60F9211242F933F9306
:101CC0004F935F936F937F938F939F93AF93BF9344
:101CD000EF93FF938091E10082FF0BC08091E200BF
:101CE00082FF07C08091E1008B7F8093E1000E941A
:101CF000C0108091DA0080FF1FC08091D80080FF63
:101D00001BC08091DA008E7F8093DA008091D90029
:101D100080FF0DC080E189BD82E189BD09B400FE6C
:101D2000FDCF81E08093F1010E94BB0A05C019BC80
:101D30001092F1010E94C90A8091E10080FF19C050
:101D40008091E20080FF15C08091E2008E7F809339
:101D5000E2008091E20080618093E2008091D800EF
:101D600080628093D80019BC85E08093F1010E94C5
:101D7000CD0A8091E10084FF30C08091E20084FFB1
:101D80002CC080E189BD82E189BD09B400FEFDCF90
:101D90008091D8008F7D8093D8008091E1008F7E64
:101DA0008093E1008091E2008F7E8093E200809139
:101DB000E20081608093E2008091ED01882311F0C0
:101DC00084E007C08091E30087FD02C081E001C08C
:101DD00083E08093F1010E94CF0A8091E10083FFAC
:101DE00029C08091E20083FF25C08091E100877FB8
:101DF0008093E10082E08093F1011092ED018091E7
:101E0000E1008E7F8093E1008091E2008E7F8093DD
:101E1000E2008091E20080618093E20042E060E0B5
:101E200080E00E94580D8091F00088608093F0005F
:101E30000E94CC0AFF91EF91BF91AF919F918F913A
:101E40007F916F915F914F913F912F910F900FBEB6
:101E50000F901F9018951F920F920FB60F9211249A
:101E60002F933F934F935F936F937F938F939F93A2
:101E7000AF93BF93CF93DF93EF93FF93C091E900AC
:101E8000CF708091EC00D82FD17080FDD0E81092F7
:101E9000E9008091F000877F8093F00078940E94A1
:101EA0006F0F1092E9008091F00088608093F0003D
:101EB000CD2BCF70C093E900FF91EF91DF91CF91CF
:101EC000BF91AF919F918F917F916F915F914F9152
:101ED0003F912F910F900FBE0F901F9018951F9359
:101EE000CF93DF93CDB7DEB7AA970FB6F894DEBFD6
:101EF0000FBECDBFE2EFF1E088E08E0F9091F100D0
:101F000091938E13FBCF0E94EB0A8091E80083FF30
:101F10001FC18091F2019091F301492F50E04A30A6
:101F2000510508F015C1FA01E15AFF4F0C945A24EB
:101F3000803881F0823809F00BC18091F6018F70F2
:101F40008093E9008091EB0085FB882780F910924F
:101F5000E90006C08091EE019091EF01911182603D
:101F60009091E800977F9093E8008093F1001092A1
:101F7000F100C8C0282F2D7F09F0EAC0882319F08E
:101F8000823061F0E5C08091F401813009F0E0C059
:101F9000933009F080E08093EF012BC08091F40131
:101FA000811127C08091F6018F7009F4D1C0809310
:101FB000E9002091EB0020FF1CC0933021F48091B8
:101FC000EB00806214C09091EB0090619093EB0065
:101FD00021E030E0A90102C0440F551F8A95E2F7C5
:101FE0004093EA001092EA008091EB0088608093B1
:101FF000EB001092E9008091E800877F86C0811194
:10200000A7C01091F4011F778091E3008078812BA5
:102010008093E3008091E800877F8093E8000E942E
:102020008D0D8091E80080FFFCCF8091E3008068F7
:102030008093E300111102C082E001C083E080932D
:10204000F10186C08058823008F082C08091F4018E
:102050009091F5018C3D53E0950779F583E08A83F3
:102060008AE289834FB7F894DE01139620E03EE0C0
:1020700051E2E32FF0E050935700E49120FF03C0BA
:10208000E295EF703F5FEF708E2F90E0EA3010F036
:10209000C79601C0C0968D939D932F5F243149F759
:1020A0004FBF8091E800877F8093E8006AE270E08C
:1020B000CE0101960E94940C14C0AE014F5F5F4F99
:1020C0006091F6010E94DB0BBC01009709F440C04F
:1020D0009091E800977F9093E80089819A810E940F
:1020E000F70C8091E8008B778093E80031C080384E
:1020F00079F58091E800877F8093E8008091ED0179
:102100008093F1008091E8008E778093E8000E9430
:102110008D0D1EC081111CC09091F4019230C0F44D
:102120008091E800877F8093E8009093ED010E9402
:102130008D0D8091ED01811106C08091E30087FD36
:1021400002C081E001C084E08093F1010E94D70ABF
:102150008091E80083FF0AC08091E800877F809328
:10216000E8008091EB0080628093EB00AA960FB6A6
:10217000F894DEBF0FBECDBFDF91CF911F910895C0
:102180000895CF938091F1018823A1F0C091E900D7
:10219000CF709091EC00892F817090FD80E8C82B62
:1021A0001092E9008091E80083FD0E946F0FCF70CC
:1021B000C093E900CF9108959093750180937401C5
:1021C0000895E0917401F0917501309721F001902C
:1021D000F081E02D099480E00895E0917401F09180
:1021E0007501309721F00280F381E02D0994089564
:1021F000E0917401F0917501309721F00480F58130
:10220000E02D099408952091720130917301821795
:10221000930771F09093730180937201E0917401C0
:10222000F0917501309721F00680F781E02D099437
:10223000089520917001309171018217930771F018
:102240009093710180937001E0917401F091750198
:10225000309721F00084F185E02D099408950895C8
:102260000C942F110E94391C0E941A040C94FB1C20
:102270009F92AF92BF92CF92DF92EF92FF920F9315
:102280001F93CF93DF9300D000D000D0CDB7DEB73F
:102290000E9432040DE010E0AA24A394B12C902EE9
:1022A000802F0E942005980129583E4F6901F901AD
:1022B000F080F826A1F40150110988F78FEF898387
:1022C0008A831B820E94421C8160782F9D838C83AD
:1022D00049815A816B818D810E94CF112FC09091CD
:1022E000DA0191FF04C08E830E9426058E8125E0CD
:1022F00030E0A501022E01C0440F0A94EAF7E42E53
:102300004F21C1F029839A828E2191E009F490E057
:102310009B830E94421C8160782F9D838C8349811E
:102320005A816B818D810E94CF11F6018081E82650
:10233000E08204C021503109E0F6BDCF0E94E21FC7
:10234000109176010E94E1101817B9F00E94E11077
:102350008093760126960FB6F894DEBF0FBECDBFF0
:10236000DF91CF911F910F91FF90EF90DF90CF9071
:10237000BF90AF909F900C94DA0926960FB6F89410
:10238000DEBF0FBECDBFDF91CF911F910F91FF90A8
:10239000EF90DF90CF90BF90AF909F900895CF9334
:1023A000DF93CDB7DEB72B970FB6F894DEBF0FBE25
:1023B000CDBF4F83588769877A878B87DE01119657
:1023C00086E0FD0111928A95E9F785E0FE013796D6
:1023D00001900D928A95E1F749815A816B817C8148
:1023E0008D819E810E9418182B960FB6F894DEBF3F
:1023F0000FBECDBFDF91CF910895CF93882309F40D
:10240000C2C0C82F823859F40E94E11081FDBBC0C0
:1024100089E30E94F21A0E94BF1B89E30CC0833833
:1024200079F40E94E11080FDAEC083E50E94F21AAB
:102430000E94BF1B83E50E94341BCF910C94BF1BED
:10244000843859F40E94E11082FD9DC087E40E9407
:10245000F21A0E94BF1B87E4EECF8CEF8C0F813AFB
:1024600048F48C2F0E94252281118DC08C2F0E9450
:10247000F21AE3CF80E28C0F883048F4C77081E015
:1024800001C0880FCA95EAF70E94781BD6CF8BE56A
:102490008C0F833078F4C53A29F0C63A31F083E8DE
:1024A00090E005C081E890E002C082E890E0CF9122
:1024B0000C94031188E58C0F833108F064C0C83A8E
:1024C00039F1C93A41F1CA3A49F1CB3A51F1CC3A22
:1024D00059F1CD3A61F1C03B69F1CE3A71F1CF3A91
:1024E00079F1C13B81F1C23B89F1C33B91F1C43B1E
:1024F00099F1C53BA1F1C63BA9F1C73BB1F1C83B7E
:10250000B9F1C93BC1F1CA3BC9F180E090E038C0E4
:1025100082EE90E035C089EE90E032C08AEE90E025
:102520002FC085EB90E02CC086EB90E029C087EBB4
:1025300090E026C08CEC90E023C08DEC90E020C0B1
:1025400083E891E01DC08AE891E01AC082E991E039
:1025500017C084E991E014C081E292E011C083E2E7
:1025600092E00EC084E292E00BC085E292E008C0E7
:1025700086E292E005C087E292E002C08AE292E041
:10258000CF910C941911CF910895882309F44BC071
:10259000823859F40E94E11081FF45C089E30E940E
:1025A000F21A0E94BF1B89E30CC0833871F40E94A9
:1025B000E11080FF38C083E50E94F21A0E94BF1B21
:1025C00083E50E94341B0C94BF1B843859F40E948D
:1025D000E11082FF28C087E40E94F21A0E94BF1B0C
:1025E00087E4EFCF9CEF980F913A58F390E2980F61
:1025F000983050F4877091E001C0990F8A95EAF7FE
:10260000892F0E947E1BDFCF9BE5980F933020F42B
:1026100080E090E00C940311885A833120F480E02C
:1026200090E00C9419110895882321F00E94781BE2
:102630000C94BF1B0895882321F00E947E1B0C94EC
:10264000BF1B08957F928F929F92AF92BF92CF92BD
:10265000DF92EF92FF920F931F93CF93DF931F921E
:10266000CDB7DEB77C01C62E772EFC010581029521
:102670000F70128111110E94951B0E94EB1A882382
:1026800079F0112369F080E28C0D883048F082E007
:102690000E94D41A0E94EB1A91E0D82ED92601C0CC
:1026A000D12CE72DE295EF70F0E0E759FF4F0C9445
:1026B0005A24872D807F072D0F70882311F00295F3
:1026C000007F112389F0002309F490C180E28C0D72
:1026D000883020F4802F0E94781B03C0802F0E9436
:1026E000881B0E94BF1B82C18C2D0E94C512002333
:1026F00009F495C180E28C0D883020F4802F0E946F
:102700007E1B03C0802F0E948E1B0E94BF1B87C1AF
:10271000972D907F872D8F70903211F08295807F5A
:10272000CC2021F0F1E0CF16B1F01EC0112349F00A
:10273000002309F414C1013009F011C10E94A81B43
:102740006EC1002319F0013009F469C189830E9428
:10275000AB1B89810AC1112321F0023008F05FC14F
:10276000FEC001115CC101C1112321F0002309F455
:10277000F6C03CC1002309F4F8C03EC1872D869500
:102780008695837090E0009719F0019761F047C13A
:10279000112321F08C2D972D937002C080E090E0E2
:1027A0000E9403113CC1112321F08C2D972D9370B1
:1027B00002C080E090E00E94191131C18C2D1123DC
:1027C00019F00E94EA1E02C00E94521F0E94D71FE9
:1027D00026C1872D837009F052C0111120C18C2DA4
:1027E000829586958770880F880F9C2D9F70892E03
:1027F000912CA12CB12C082E04C0880C991CAA1C69
:10280000BB1C0A94D2F7C4FE14C00FE010E020E015
:1028100030E0B901A80104C0440F551F661F771F9F
:102820008A95D2F7CB01BA01609570958095909505
:1028300003C060E070E0CB01272D2695269523701C
:1028400030E02230310569F02330310589F0682904
:1028500079298A299B292130310571F00E9460195C
:10286000DEC0682979298A299B290E947C19D7C052
:102870000E946019C501B4010E944419D0C01123FF
:1028800019F0872D817001C08695882309F4C7C08F
:102890008C2D829586958770880F880F9C2D9F7050
:1028A000892E912CA12CB12C082E04C0880C991CC7
:1028B000AA1CBB1C0A94D2F7C4FE14C00FE010E09F
:1028C00020E030E0B901A80104C0440F551F661F85
:1028D000771F8A95D2F7CB01BA01609570958095E4
:1028E000909503C060E070E0CB01272D26952695DA
:1028F0002370422F50E04230510569F043305105BA
:1029000089F0682979298A299B294130510571F07C
:102910000E943A1A84C0682979298A299B290E9431
:10292000561A7DC00E943A1AC501B4010E941E1AAF
:1029300076C08C2D90E0FC01E05EF109E531F105F7
:1029400008F050C0E758FF4F0C945A240C2D0F701C
:10295000872D8F71112331F00E94B719802F0E94AB
:1029600014135DC00E94D819802F0E941B1357C0FA
:10297000112339F0011153C0872D8F710E94FD1969
:102980004EC0023008F04BC0F7CF112339F0872D2D
:102990008F710E94B71943C01123C9F3872D8F711E
:1029A0000E94D8193CC0112329F0872D8F710E94F5
:1029B000A21935C00E94981932C0112351F0172D69
:1029C0001F71812F0E94B71963E0812F0E94CB1ADB
:1029D00026C081E00E94D41A023008F182E00E94F1
:1029E000D41A1DC0112331F0002389F28C2D0E94CE
:1029F000FD1115C0002391F28C2D0E94C5120FC04D
:102A0000472D4F706C2DC7010E94FE050E94BC1817
:102A100006C0472D4F706C2DC7010E94E906DD20CE
:102A2000F9F00E94C71A80FD1BC0F70112820E94B4
:102A3000C11A0E94B719C7010E943F150E94C11A0E
:102A40000F90DF91CF911F910F91FF90EF90DF904A
:102A5000CF90BF90AF909F908F907F900C94D8199B
:102A60000F90DF91CF911F910F91FF90EF90DF902A
:102A7000CF90BF90AF909F908F907F9008950F93CD
:102A80001F93CF93DF93EC01888199812B813C8147
:102A9000232BB9F09F3F11F48F3F99F0CE010E9494
:102AA0004106882371F0688179818A810E94BD1A6C
:102AB0008C010E94721A0E943919B801CE010E943D
:102AC0002213DF91CF911F910F9108950E94951BC2
:102AD0000E94A51B0E946A1B0E94BF1B0E948820A7
:102AE0000E94D71F80E090E00E94031180E090E0F8
:102AF0000C9419110E94851B0C9466150E94B21A41
:102B0000292F22952F7030E02C3031054CF42A30DB
:102B100031056CF42250310922303105A8F407C088
:102B20002C30310569F02F30310551F00DC0803F58
:102B300069F018F4803E40F409C0843F29F406C0CF
:102B400093FB882780F9089580E0089581E0089537
:102B5000CF93DF9300D000D01F92CDB7DEB70F9098
:102B60000F900F900F900F90DF91CF910895CF931A
:102B7000DF9300D000D000D0CDB7DEB726960FB6D9
:102B8000F894DEBF0FBECDBFDF91CF9108951F93A4
:102B9000CF93DF93C091850116E080918601C8171D
:102BA00099F0D0E01C9FF0011D9FF00D1124E95712
:102BB000FE4F4081518162817381848195810E94A1
:102BC000B7152196C770E9CFDF91CF911F91089576
:102BD0004091B7015091B8016091B9017091BA016B
:102BE0008091BB019091BC010C94B7158091BC0100
:102BF00082958F7009F054C08091B901882309F43F
:102C00004FC080918501A09186016091B7017091BC
:102C1000B8014091BA015091BB01B6E08A1709F49E
:102C20003FC090E041155105C1F17F3F11F46F3F66
:102C3000A1F1B89FF001B99FF00D1124E957FE4FA3
:102C4000218172132AC02081621327C022812111A1
:102C500024C0238134812417350710F42150310911
:102C6000241B350B283C3105C0F42091BC012F708A
:102C700020612093BC0126E0289FF001299FF00DE0
:102C80001124E457FE4F80818F708061808387EB31
:102C900091E00E943F150C94C71501968770BECF36
:102CA0000895CF92DF92EF92FF920F931F93CF93ED
:102CB000DF93CDB7DEB762970FB6F894DEBF0FBED5
:102CC000CDBF8C0185E0F801DE011D9601900D92CB
:102CD0008A95E1F7D8014C9111965C911197129663
:102CE0006C9112971396CD90DC9014973091B701A8
:102CF0007091B8018091BA019091BB01009709F4DD
:102D00006BC17F3F19F43F3F09F466C1E090B90100
:102D1000EE2009F4C0C02091BC01C816D90628F0E5
:102D2000F601E81BF90BCF0104C0809590958C0D3E
:102D30009D1DFF24F394883C910578F0F12C207FB1
:102D400009F0C6C07C2DD98AC88A89890E94A81535
:102D500087EB91E00E943F15B1C0822F807F09F080
:102D600046C0751314C0341312C0611110C02F7007
:102D700020612093BC010E94E81587EB91E00E943E
:102D80003F158091BC01D80115968C932EC0CD289B
:102D900019F15F3F11F44F3FF9F0F62E61111CC09D
:102DA000809185012091860136E0821709F45AC08E
:102DB00090E0389FF001399FF00D1124E957FE4F44
:102DC0007181571306C07081471303C0728171115E
:102DD00003C001968770E9CFF62E662309F418C167
:102DE0008091BC0181608093BC01F12C11C17513ED
:102DF00008C0341306C0611104C08091BC01D80121
:102E0000C3C04D875E878D859E856A8B0E947E1527
:102E10006A898823E1F16623D1F12091BC01822FD8
:102E200082958F7090E0029774F08091B701909135
:102E3000B80198878F831986DB86CA862C87CE01D6
:102E400007960E943F1586E0F801A7EBB1E00190DC
:102E50000D928A95E1F70E94F6150E94E815FF246D
:102E6000F394D6C04D875E878D859E850E94B21AE9
:102E7000292F22952F7030E0223031050CF0BCC094
:102E80009F7009F0B6C0805E883008F4C1C0C801E8
:102E90000E943F15E4CFC816D90608F453C0F601C6
:102EA000E81BF90BCF01883C910508F450C0F12CC8
:102EB0007C2DD98AC88A89890E94A815E7EBF1E0A0
:102EC00086E0DF011D928A95E9F70E94E815A0C00F
:102ED000751314C0341312C0611110C08091BC016D
:102EE000F8018583C8010E943F1586E0E7EBF1E019
:102EF000DF011D928A95E9F7FE2C8AC04D875E8717
:102F00008D859E856A8B0E947E156A89882309F4C7
:102F1000BECF662309F4BBCF2091BC01822F8295DE
:102F20008F7090E002970CF48ECF8091B701909152
:102F3000B8019A8389831B82DD82CC822E83CE01E5
:102F400001967FCF809590958C0D9D1DACCFF62E70
:102F5000662309F49CCF75132EC034132CC0209126
:102F6000BC0120FD1FC0822F82958F70D9F0D8013F
:102F700015962C9315978F3049F08F5F982F929567
:102F8000907F822F8F70892B15968C93C8010E9499
:102F90003F1586E0F801A7EBB1E001900D928A950C
:102FA000E1F793CF86E0F801A7EBB1E001900D9235
:102FB0008A95E1F72DC04D875E878D859E850E949D
:102FC0007E15811140CF8091BC0181608093BC014E
:102FD000C8010E943F151CC0662309F458CF4D87D5
:102FE0005E878D859E850E947E15882309F44FCFCC
:102FF0002ACF811148CF0CC0243031050CF047CFC7
:103000009F7009F440CFF8019581907F09F03BCF84
:103010008F2D62960FB6F894DEBF0FBECDBFDF9145
:10302000CF911F910F91FF90EF90DF90CF90089577
:103030001F93CF93DF93CDB7DEB72C970FB6F894DD
:10304000DEBF0FBECDBF4F83588769877A878B87D6
:103050009C87CE0107960E945116882369F08F81C4
:1030600098852A853B85232BF1F19F3F09F063C0AA
:103070008F3F09F060C037C086E0FE013796DE0161
:10308000119601900D928A95E1F76F817885EA8516
:10309000FB85309741F17F3F11F46F3F21F1209183
:1030A000860130E0C901019687709927409185011A
:1030B00050E08417950709F447C069837A83FD833C
:1030C000EC8396E0929FD001939FB00D1124A957F5
:1030D000BE4FFE01319601900D929A95E1F78093D3
:1030E00086010E94C71516E08091850190918601A6
:1030F0008917C1F1189FC001112489579E4F0E9462
:103100005116882379F1E09185011E9FF001112469
:10311000E957FE4F4081518162817381848195819D
:103120000E94B7158091850190E0019687709927DC
:1031300080938501D9CF4F81588569857A858B85A4
:103140009C850E94B715CFCF0E947A1510928601F8
:1031500010928501E7EBF1E086E0DF011D928A9590
:10316000E9F7C1CF2C960FB6F894DEBF0FBECDBFE6
:10317000DF91CF911F910895EF92FF920F931F93CC
:10318000CF93DF938C01009709F46CC0F12CEE24EF
:10319000E394E8012196F8018491843740F4843067
:1031A00008F051C0813081F0823019F15BC0853761
:1031B00009F444C0A8F19CE7980F903708F052C07A
:1031C0008F770E94C51241C00E5F1F4FFE01C49150
:1031D00080E28C0F883048F4C7708E2D01C0880FB4
:1031E000CA95EAF70E94981B14C08C2F0E94FD110B
:1031F0002DC00E5F1F4FFE01C49180E28C0F8830FE
:1032000058F4C7708E2D01C0880FCA95EAF70E9446
:103210009E1B0E94BF1B1AC08C2F0E94C51216C095
:103220000E5F1F4FFE01C491CC2381F08FE99FE018
:103230000197F1F700C00000C150F6CF0E5F1F4F9D
:10324000FE01F49003C00E94FD118E018F2D882392
:1032500009F49FCFEFE9FFE03197F1F700C00000DC
:103260008150F5CFDF91CF911F910F91FF90EF909B
:10327000089508956093C1017093C2018093C301C2
:103280009093C4010C9466150F931F930091C10194
:103290001091C2012091C3013091C401DC01CB0126
:1032A000802B912BA22BB32B8093C1019093C20151
:1032B000A093C301B093C4011F910F910C946615A4
:1032C0000F931F930091C1011091C2012091C3017E
:1032D0003091C401DC01CB0180239123A223B323CD
:1032E0008093C1019093C201A093C301B093C40124
:1032F0001F910F910C9466150F931F930091C101BC
:103300001091C2012091C3013091C401DC01CB01B5
:1033100080279127A227B3278093C1019093C201F0
:10332000A093C301B093C4011F910F910C94661533
:103330001092BD011092BE011092BF011092C00107
:103340000C94661541E050E060E070E004C0440F6A
:10335000551F661F771F8A95D2F74093BD01509382
:10336000BE016093BF017093C0010C94661541E0EB
:1033700050E060E070E004C0440F551F661F771FE7
:103380008A95D2F78091BD019091BE01A091BF01B5
:10339000B091C001482B592B6A2B7B2B4093BD0168
:1033A0005093BE016093BF017093C0010C946615E9
:1033B00041E050E060E070E004C0440F551F661F1C
:1033C000771F8A95D2F740955095609570958091BA
:1033D000BD019091BE01A091BF01B091C0014823F1
:1033E00059236A237B234093BD015093BE01609310
:1033F000BF017093C0010C94661541E050E060E09D
:1034000070E004C0440F551F661F771F8A95D2F7DE
:103410008091BD019091BE01A091BF01B091C0010A
:10342000482759276A277B274093BD015093BE0147
:103430006093BF017093C0010C9466150F931F93A6
:103440000091BD011091BE012091BF013091C001DA
:10345000DC01CB01802B912BA22BB32B8093BD01E0
:103460009093BE01A093BF01B093C0011F910F9133
:103470000C9466150F931F930091BD011091BE012E
:103480002091BF013091C001DC01CB018023912349
:10349000A223B3238093BD019093BE01A093BF01EB
:1034A000B093C0011F910F910C9466150F931F9359
:1034B0000091BD011091BE012091BF013091C0016A
:1034C000DC01CB0180279127A227B3278093BD0180
:1034D0009093BE01A093BF01B093C0011F910F91C3
:1034E0000C9466150895CF92DF92EF92FF920F939E
:1034F0001F93CF93DF938C01C090C101D090C20184
:10350000E090C301F090C4018091BD019091BE0193
:10351000A091BF01B091C001C82AD92AEA2AFB2A8A
:10352000CFE1D0E0D701C6010C2E04C0B695A79517
:10353000979587950A94D2F780FF06C0B8018C2F23
:103540000E943F09019721F4219760F780E001C0B4
:103550008C2FDF91CF911F910F91FF90EF90DF9013
:10356000CF900895CF93DF93EC010E94731ABE01B0
:103570000E943F09DF91CF910895CB010E94B21ABA
:1035800008958091C50185958595859508958091CB
:10359000C5018770089598E0899F90011124262B1A
:1035A0002093C5010C94B7192091C5018095822301
:1035B0008093C501982F977069F430E0482F552704
:1035C00047FD50952417350729F0859585958595F4
:1035D0000C94D81908959091C501977081E009F471
:1035E00080E0089590910C01992321F090910D01B4
:1035F000911109C020910E0130910F01F90132960D
:103600009FEF40E01FC0982F9695969596959F3016
:1036100050F5E0910E01F0910F01E90FF11D877057
:1036200021E030E0A90102C0440F551F8A95E2F75E
:10363000CA019181892B818308959F3F39F04F5FA3
:103640004E3041F051915813F8CF0DC05111F7CFC2
:10365000942FF5CF9F3F39F0F901E90FF11D97FD48
:10366000FA9582830895089590910C01992321F091
:1036700090910D01911109C020910E0130910F011F
:10368000F9013296205F3F4F1FC0982F969596956F
:1036900096959F30F0F4E0910E01F0910F01E90F43
:1036A000F11D877021E030E0A90102C0440F551FD1
:1036B0008A95E2F7CA0180959181892381830895D3
:1036C0003196E217F30729F090819813F9CF108211
:1036D000F7CF089581E090E0E0910E01F0910F01A5
:1036E000E80FF91F1082019680319105A9F708951E
:1036F0009091D901892B8093D9010895809590915B
:10370000D90189238093D90108951092D901089590
:103710009091D801892B8093D8010895809590913C
:10372000D80189238093D80108951092D801089573
:103730009091D701892B8093D7010895809590911E
:10374000D70189238093D70108951092D701089556
:103750008093C60108951092C601089580910E01CC
:1037600090910F01FC0131969C01205F3F4F80E05A
:10377000919191118F5FE217F307D1F70895E091CE
:103780000E01F0910F018091D9018083E0910E012B
:10379000F0910F0190818091D801892B8083E09175
:1037A0000E01F0910F0190818091D701892B8083C8
:1037B0008091C601882361F0E0910E01F0910F0124
:1037C0009081892B80830E94AE1B81111092C601CB
:1037D00080910E0190910F010C94ED1020E0009764
:1037E00039F0AC0141505109842395232F5FF7CF65
:1037F000822F08958091F101843021F11092DB0134
:1038000020E488E190E00FB6F894A89580936000DA
:103810000FBE2093600080E00E94DA0983B7817FA9
:10382000846083BF83B7816083BF7894889583B7B2
:103830008E7F83BF88E10FB6F8948093600010926A
:1038400060000FBE0895089508950E94231C0E94F1
:1038500032040E94241C0E94270591E0811101C0BE
:1038600090E0892F08950E947A150E94E1100C942F
:10387000DA0982E084BD93E095BD9AEF97BD80930D
:103880006E0008952FB7F8948091DC019091DD01CE
:10389000A091DE01B091DF012FBF0895CF92DF929A
:1038A000EF92FF920F931F932FB7F8944091DC0192
:1038B0005091DD016091DE017091DF012FBF6A013F
:1038C0007B01EE24FF248C0120E030E0C016D106FD
:1038D000E206F30610F4415051099A01281B390BF6
:1038E000C9011F910F91FF90EF90DF90CF90089545
:1038F0001F920F920FB60F9211248F939F93AF9345
:10390000BF938091DC019091DD01A091DE01B09127
:10391000DF010196A11DB11D8093DC019093DD01B3
:10392000A093DE01B093DF01BF91AF919F918F9182
:103930000F900FBE0F901F9018950E94DE0DF89407
:103940002FEF87EA91E6215080409040E1F700C0D8
:10395000000087E090EBDC018093FB019093FC0179
:10396000A093FD01B093FE019CE088E10FB6F894AE
:10397000A895809360000FBE90936000FFCFEF92F8
:10398000FF920F931F93CF93DF93D82FCDE08C2F0F
:103990000E94200505E010E0E82EF12CC701002E62
:1039A00002C0959587950A94E2F780FF09C0602FC1
:1039B0007C2F80E00E94EA06D81302C081E006C096
:1039C0000150110958F7C15010F780E0DF91CF91F5
:1039D0001F910F91FF90EF900895CF93C82F8CE225
:1039E0000E94BF1C882321F08C2FCF910C94BF1C08
:1039F00080E0CF910895CF930E94421E811102C0B2
:103A00000E94281EC5E6C15049F00E9432048FE38F
:103A10009CE90197F1F700C00000F5CF89E20E9410
:103A2000ED1C811113C18AE20E94ED1C81110E94DC
:103A3000281E85E00E94ED1C81110E949D1C0E94A1
:103A40004D1E8093DA0187E00E94ED1C8823A9F1C6
:103A50008BE10E94ED1C882351F08091DA0181FBFB
:103A6000222720F991E0922790FB81F90EC08EE089
:103A70000E94ED1C882361F08091DA0182FB2227ED
:103A800020F991E0922790FB82F98093DA0115C02A
:103A900080E10E94ED1C9091DA01882341F093FBB4
:103AA000222720F981E0822780FB93F904C0892F27
:103AB000809580FB90F99093DA018091DA010E9461
:103AC000511E0E945F1E8093FA0180EE0E94ED1C41
:103AD000882341F08091FA01982F909590FB80F90E
:103AE0008093FA0189E30E94ED1C882359F08091AC
:103AF000FA0181FB222720F991E0922790FB81F9BE
:103B00008093FA0182EE0E94ED1C882359F0809187
:103B1000FA0182FB222720F991E0922790FB82F99B
:103B20008093FA0186EE0E94ED1C882359F0809163
:103B3000FA0183FB222720F991E0922790FB83F979
:103B40008093FA0183EE0E94ED1C882359F0809146
:103B5000FA0184FB222720F991E0922790FB84F957
:103B60008093FA0185E30E94ED1C882359F080912F
:103B7000FA0185FB222720F991E0922790FB85F935
:103B80008093FA0181E30E94ED1C882359F0809113
:103B9000FA0186FB222720F991E0922790FB86F913
:103BA0008093FA0181E10E94ED1C882359F08091F5
:103BB000FA0187FB222720F991E0922790FB87F9F1
:103BC0008093FA018091FA010E94631E8091FA01AC
:103BD00087FB882780F980930D0187E20E94ED1C06
:103BE000C82F8EE10E94ED1C8111C2608FE10E94FE
:103BF000ED1C8111C46080E20E94ED1C8111C8603F
:103C000081E20E94ED1C8111C06182E20E94ED1CE4
:103C10008111C06283E20E94ED1C8111C06484E2C4
:103C20000E94ED1C882311F0C06802C0CC2329F04B
:103C30008C2F0E945A1E6C2F03C00E94561E682FA4
:103C400070E080E090E0CF910C943A19CF91089504
:103C50006DEE7EEF80E090E00E94942460E082E0D0
:103C600090E00E94822460E083E090E00E94822441
:103C700060E084E090E00E94822460E085E090E0D3
:103C80000C94822480E090E00E947C2421E08D3E10
:103C90009E4F09F020E0822F089582E090E00C947E
:103CA0007424682F82E090E00C94822483E090E0FA
:103CB0000C947424682F83E090E00C94822484E0B8
:103CC00090E00C947424682F84E090E00C9482249B
:103CD0008091E20180FF0BC06091130185E0689F35
:103CE000B001112475956795759567952BC081FF77
:103CF00009C06091130185E0689FB001112475959A
:103D0000679520C082FF07C06091130185E0689F1E
:103D1000B001112417C09091E3019923D1F0609173
:103D20001201961788F72091130185E0289F9001D2
:103D30001124929FA001939F500D112470E0CA019D
:103D40000E9446246038710540F46115710539F010
:103D500002C065E070E0862F08958FE7089581E046
:103D600008958091E20180FF08C06091110170E028
:103D7000759567957595679521C081FF06C060911F
:103D8000110170E07595679519C082FF04C06091BC
:103D9000110170E010C09091E3019923C1F060918E
:103DA00010019617A0F780911101899FC00111247D
:103DB00070E00E9446246038710528F46115710591
:103DC00021F0862F08958FE7089581E0089561E03E
:103DD00070E0F4CF803F21F40E94681E819504C0FA
:103DE000813F29F40E94681E8093E6010895823F76
:103DF00021F40E94681E819504C0833F29F40E942B
:103E0000681E8093E5010895893F19F40E94B11E50
:103E100005C08A3F31F40E94B11E81958093E7016D
:103E200008958B3F21F40E94B11E819504C08C3F00
:103E300029F40E94B11E8093E8010895843F21F483
:103E40008091E401816017C0853F21F48091E401F5
:103E5000826011C0863F21F48091E40184600BC030
:103E6000873F21F48091E401886005C0883F31F4E8
:103E70008091E40180618093E40108958D3F21F4F5
:103E80008091E20181600BC08E3F21F48091E201BC
:103E9000826005C08F3F29F48091E20184608093A5
:103EA000E2010895803F39F48091E60187FF6CC0FC
:103EB0001092E60169C0813F29F48091E60118164D
:103EC000BCF362C09091E501823F29F497FF5CC08A
:103ED0001092E50159C0833F19F41916CCF354C070
:103EE000893F41F48091E70118160CF04DC0109203
:103EF000E7014AC08A3F29F48091E70187FF44C067
:103F0000F6CF8B3F39F48091E80187FF3DC01092D6
:103F1000E8013AC08C3F29F48091E8011816BCF3FF
:103F200033C0843F21F48091E4018E7F17C0853F28
:103F300021F48091E4018D7F11C0863F21F48091AE
:103F4000E4018B7F0BC0873F21F48091E401877FE0
:103F500005C0883F31F48091E4018F7E8093E401B5
:103F600013C08D3F21F48091E2018E7F0BC08E3F04
:103F700021F48091E2018D7F05C08F3F29F480916B
:103F8000E2018B7F8093E2018091E50181110EC0F7
:103F90008091E60181110AC08091E701811106C07C
:103FA0008091E801811102C01092E301089584EE2E
:103FB00091E00E94F8100E94421C9093E1018093CE
:103FC000E00108951F93CF93DF938091E0019091DA
:103FD000E1010E944E1CAC019091E301992321F074
:103FE0002091140130E006C0209115018AE0289F3D
:103FF000900111244217530708F486C08091E5010F
:10400000C091E601D091E7011091E801811107C04C
:10401000C11176C0D11174C0111172C075C09F3F1B
:1040200019F09F5F9093E301181624F40E94681E14
:104030008093E5018091E50187FF05C00E94681E1D
:1040400081958093E5011C1624F40E94681E8093DC
:10405000E6018091E60187FF05C00E94681E8195F8
:104060008093E6016091E501662339F1C091E60194
:10407000CC2319F1772767FD7095872F972F0E9422
:10408000572323E333E343E35FE30E94BB230E9410
:1040900024236093E5016C2F772767FD7095872FA8
:1040A000972F0E94572323E333E343E35FE30E9408
:1040B000BB230E9424236093E6011D1624F40E9472
:1040C000B11E8093E7018091E70187FF05C00E9440
:1040D000B11E81958093E701111624F40E94B11E50
:1040E0008093E8018091E80187FF05C00E94B11E1E
:1040F00081958093E801DF91CF911F910C94D71F98
:104100009F3F09F08ECF96CFDF91CF911F910895F9
:10411000E4EEF1E085E0DF011D928A95E9F7109267
:10412000E3011092E2010895833081F128F4813097
:1041300059F08230D1F00895853009F449C0B8F1C2
:10414000863009F456C0089580911501262F30E07D
:10415000280F311D2F3F310524F4680F609315019E
:1041600008958FEF80931501089580911401262FF3
:1041700030E0280F311D2F3F310524F4680F609384
:10418000140108958FEF8093140108958091130115
:10419000262F30E0280F311D2F3F310524F4680F02
:1041A0006093130108958FEF809313010895809118
:1041B0001201262F30E0280F311D2F3F310524F446
:1041C000680F6093120108958FEF80931201089594
:1041D00080911101262F30E0280F311D2F3F31052E
:1041E00024F4680F6093110108958FEF80931101FB
:1041F000089580911001262F30E0280F311D2F3FA8
:10420000310524F4680F6093100108958FEF8093B7
:1042100010010895833011F128F4813049F0823083
:1042200091F00895853081F120F18630C1F1089533
:1042300080911501681720F4861B8093150108955D
:1042400010921501089580911401681720F4861BBF
:104250008093140108951092140108958091130120
:10426000681720F4861B80931301089510921301A0
:10427000089580911201681720F4861B8093120123
:10428000089510921201089580911101681720F489
:10429000861B809311010895109211010895809159
:1042A0001001681720F4861B809310010895109266
:1042B000100108950F931F938D3109F46BC008F01E
:1042C0003FC08E3009F47FC0C0F4873009F469C064
:1042D00068F4863009F0B1C08091DA01817F8E7F69
:1042E0008093DA0181E08093EA01A8C0883009F464
:1042F000A2C08B3009F49FC0A0C0863109F49BC0D6
:1043000078F4803109F472C0813109F096C00E94BE
:104310007A1590910D0181E0892780930D018BC062
:10432000893109F488C08B3109F087C08091DA01A6
:1043300081FB222720F991E0922790FB81F94CC064
:10434000853309F470C048F4873209F46CC008F46E
:1043500059C0893209F467C070C0833438F48A3395
:1043600008F04EC0883309F466C067C0833409F48E
:104370005AC0883409F061C00E947A150FEF13ED1E
:1043800020E3015010402040E1F700C000000E94EF
:104390009D1C51C00E94DE220E94E1100E94DA0999
:1043A0004AC09091DA01892F8095817080FB90F945
:1043B00029F0966098609093DA0140C0997F977FCA
:1043C0009093DA0138C08091DA0182FB222720F92C
:1043D00091E0922790FB82F98093DA01992359F1B9
:1043E0008091DA0181608093DA0125C08091DA0141
:1043F00083FB222720F991E0922790FB83F9ECCFF1
:10440000895301C08D5141E050E060E070E08A01C5
:104410009B0104C0000F111F221F331F8A95D2F782
:10442000C901B80104C061E070E080E090E00E9442
:104430003A190E947A1581E001C080E01F910F9126
:10444000089580E0089580E00895CF93C82F80916B
:10445000EA01813079F018F08230E9F187C0E0910B
:104460000E01F0910F018081813169F0823209F0F3
:104470007FC009C0E0910E01F0910F018081813170
:1044800011F0823261F48C2F0E942122811104C02C
:104490008C2F0E945A211DC081E090E01AC08C2F01
:1044A0000E942322811114C0C43179F048F4CB302A
:1044B00079F0C03109F060C082E08093EA0108C061
:1044C000C93219F0C83321F057C01092EA0154C024
:1044D00081E0817053C0C93289F118F5C43171F19E
:1044E000A8F4C73009F046C08AE08093150194E132
:1044F0009093140193E0909313018093120188E04C
:104500008093110188E28093100134C0CE51C630EF
:1045100088F5EC2FF0E0E65DFE4F80818093E901A5
:1045200029C0CE34E9F020F4CB3421F56AE013C081
:10453000C13579F0C235F1F461E00DC08091E90137
:10454000882319F01092E90115C081E08093EA01F7
:1045500015C061E006C08091E9010E9494200AC064
:104560006AE08091E9010E940A2104C01092EA01E8
:1045700080E004C081E002C080E0ABCFCF9108951D
:10458000E1E8F0E0808188608083808181608083C1
:104590008FB7F89493E09093890090ED9093880002
:1045A0008FBF0895EFE6F0E08081826080830895F8
:1045B000EFE6F0E080818D7F80830895EFE6F0E004
:1045C000908182E08927808308951F920F920FB611
:1045D0000F9211242F933F934F935F936F937F9389
:1045E0008F939F93AF93BF93EF93FF938091EB01D2
:1045F0009091EC0101969093EC018093EB01811175
:1046000003C082E00E94DA09E091EC01E695E695AC
:10461000F0E0EF57F94FE4918091EB018E1303C066
:1046200080E00E94DA09FF91EF91BF91AF919F91D5
:104630008F917F916F915F914F913F912F910F904B
:104640000FBE0F901F90189504D06894B1118DC0C3
:10465000089570D088F09F5790F0B92F9927B751DF
:10466000A0F0D1F0660F771F881F991F1AF0BA9536
:10467000C9F712C0B13081F077D0B1E0089574C0AD
:10468000672F782F8827B85F39F0B93FCCF386952C
:1046900077956795B395D9F73EF490958095709589
:1046A00061957F4F8F4F9F4F0895E89409C097FB06
:1046B0003EF490958095709561957F4F8F4F9F4FF9
:1046C0009923A9F0F92F96E9BB279395F69587953D
:1046D00077956795B795F111F8CFFAF4BB0F11F400
:1046E00060FF1BC06F5F7F4F8F4F9F4F16C08823A7
:1046F00011F096E911C0772321F09EE8872F762FDD
:1047000005C0662371F096E8862F70E060E02AF01D
:104710009A95660F771F881FDAF7880F9695879509
:1047200097F9089557FD9058440F551F59F05F3F72
:1047300071F04795880F97FB991F61F09F3F79F0C3
:1047400087950895121613061406551FF2CF469545
:10475000F1DF08C0161617061806991FF1CF8695C7
:104760007105610508940895E894BB2766277727AB
:10477000CB0197F908950BD078C069D028F06ED09E
:1047800018F0952309F05AC05FC01124EECFCADF9C
:10479000A0F3959FD1F3950F50E0551F629FF00154
:1047A000729FBB27F00DB11D639FAA27F00DB11DAD
:1047B000AA1F649F6627B00DA11D661F829F222736
:1047C000B00DA11D621F739FB00DA11D621F839FBD
:1047D000A00D611D221F749F3327A00D611D231F93
:1047E000849F600D211D822F762F6A2F11249F57E1
:1047F00050408AF0E1F088234AF0EE0FFF1FBB1F04
:10480000661F771F881F91505040A9F79E3F5105A2
:1048100070F014C0AACF5F3FECF3983EDCF38695AE
:1048200077956795B795F795E7959F5FC1F7FE2B4D
:10483000880F911D9695879597F9089597F99F6729
:1048400080E870E060E008959FEF80EC0895002418
:104850000A941616170618060906089500240A94E5
:1048600012161306140605060895092E0394000C6B
:1048700011F4882352F0BB0F40F4BF2B11F460FFFA
:1048800004C06F5F7F4F8F4F9F4F089597FB072E98
:1048900016F4009407D077FD09D00E94602407FC2D
:1048A00005D03EF4909581959F4F08957095619540
:1048B0007F4F0895EE0FFF1F0590F491E02D0994AE
:1048C000AA1BBB1B51E107C0AA1FBB1FA617B70736
:1048D00010F0A61BB70B881F991F5A95A9F7809552
:1048E0009095BC01CD010895F999FECF92BD81BD8F
:1048F000F89A992780B50895A8E1B0E042E050E029
:104900000C949C24262FF999FECF92BD81BDF89A74
:10491000019700B4021639F01FBA20BD0FB6F89403
:10492000FA9AF99A0FBE08950196272F0E948324C0
:104930000C948224DC01CB01FC01F999FECF06C066
:10494000F2BDE1BDF89A319600B40D92415050404D
:08495000B8F70895F894FFCFB9
:104958000220DC096A0A470A130ADF090101C701B4
:1049680028080A03140A3F4D36394206F505BF05E3
:104978008605190532054B05640501020304050681
:044988000708090013
:00000001FF
